:10800000FEDF07EA000000000000000000000000A2
:108010000000000000000000000000000000000060
:108020000000000000000000000000000000000050
:108030000000000000000000000000000000000040
:108040000000000000000000000000000000000030
:02000004001FDB
:020000040020DA
:1000000002D3A0E3C00000EBFEFFFFEA001080E592
:100010001EFF2FE1B010C0E11EFF2FE10010C0E570
:100020001EFF2FE1000090E51EFF2FE10E00A0E172
:100030001EFF2FE110FF2FE11EFF2FE110402DE9E1
:1000400008009FE5F6FFFFEB1040BDE81EFF2FE123
:100050005450212010402DE91C009FE5F0FFFFEBDC
:10006000010010E3FBFFFF0A10009FE5ECFFFFEB30
:100070001040BDE8FF0000E21EFF2FE15450212098
:100080004050212010402DE90C009FE5E4FFFFEBDC
:100090001040BDE8010000E21EFF2FE15450212076
:1000A00010402DE90040A0E11C009FE5DCFFFFEBC4
:1000B000200010E3FBFFFF0A0410A0E10C009FE505
:1000C000D1FFFFEB1040BDE81EFF2FE1545021206F
:1000D0004050212010402DE910009FE5D0FFFFEB9C
:1000E000010C10E3FBFFFF1A1040BDE81EFF2FE1DB
:1000F0005450212070402DE90050A0E12040A0E3A1
:10010000044044E23504A0E10F0000E2090050E39E
:100110003700808230008092E0FFFFEB000054E364
:10012000F6FFFF1A2000A0E37040BDE8DBFFFFEA06
:1001300010402DE9EEFFFFEB0D00A0E3D7FFFFEB32
:100140000A00A0E31040BDE8D4FFFFEA10402DE90B
:100150000110A0E3D4009FE5ABFFFFEB0010A0E38C
:10016000CC009FE5A8FFFFEB0010A0E3C4009FE5D3
:10017000A5FFFFEB0310A0E3BC009FE5A2FFFFEB90
:100180000010A0E3B4009FE59FFFFFEB0010A0E389
:100190009C009FE59CFFFFEBC610A0E3A0009FE53D
:1001A00099FFFFEB9C109FE59C009FE596FFFFEBFE
:1001B00098009FE59AFFFFEB3F1AC0E3121A81E314
:1001C00088009FE590FFFFEB0010A0E380009FE513
:1001D0008DFFFFEB0040A0E30400A0E1014084E2BA
:1001E00094FFFFEB960054E3FAFFFF1A0319A0E314
:1001F00060009FE584FFFFEB0040A0E30400A0E166
:10020000014084E28BFFFFEB960054E3FAFFFF1AF4
:100210000010A0E33C009FE57BFFFFEB0310A0E391
:1002200010009FE578FFFFEB1040BDE81EFF2FE1B7
:100230000450212044502120605021204C50212086
:1002400050502120485021200E01000068502120EC
:1002500004002020940020209800202010402DE948
:100260001C409FE5F918A0E30400A0E166FFFFEB46
:100270000400A0E10C109FE563FFFFEB1040BDE818
:100280001EFF2FE108B400200002F90010402DE904
:1002900008009FE562FFFFEB1040BDE81EFF2FE165
:1002A00020B4002070402DE954409FE50400A0E1F7
:1002B0005BFFFFEB4C509FE50E16C0E3021681E397
:1002C0000400A0E150FFFFEB0500A0E154FFFFEBAD
:1002D0000E19C0E31C4084E20500A0E1021981E38D
:1002E00049FFFFEB0400A0E10219A0E346FFFFEB8A
:1002F0000400A0E10810A0E343FFFFEB7040BDE85D
:100300001EFF2FE1100020200C002020F0472DE9D7
:100310000080A0E3E2FFFFEB8BFFFFEB40029FE5D5
:1003200082FFFFEB40FFFFEB80FFFFEB4900A0E304
:100330005AFFFFEB4800A0E358FFFFEB4500A0E3A6
:1003400056FFFFEB5800A0E354FFFFEB0D00A0E3C6
:1003500052FFFFEB0A00A0E30890A0E10860A0E1D3
:100360000850A0E10870A0E10840A0E14BFFFFEBBE
:1003700037FFFFEB3A0050E32B00000A0D0050E37B
:100380000A00501301A0A00300A0A0132900000A36
:100390002030C0E3470053E35000000A013044E23C
:1003A000140053E303F19F97F0FFFFEA1C042000C1
:1003B0001C042000BC042000BC042000BC0420005D
:1003C000BC0420009C0420006404200040042000A1
:1003D0004004200040042000400420003404200099
:1003E000000420000004200000042000000420007D
:1003F000000420000004200000042000000420006D
:10040000390050E3070040820992A0E10F0000E2AA
:10041000150054E3099080E14500000A0CFFFFEB52
:100420003A0050E3014084E2D3FFFF1A0140A0E309
:10043000CEFFFFEA0662A0E10040A0E3CBFFFFEAA7
:10044000390050E3070040820662A0E10F0000E29D
:10045000066080E10668A0E12668A0E1014084E230
:10046000C2FFFFEA390050E3070040820552A0E1D5
:100470000F0000E2055080E1FF5005E2010055E366
:100480002700000A0E40A033B8FFFF3A020055E3F0
:100490000940A0030040A013B4FFFFEA390050E375
:1004A000070040820552A0E10F0000E2055080E104
:1004B000FF5005E20840A0E3ACFFFFEA390050E33B
:1004C000070040820772A0E10F0000E2077080E1A0
:1004D0000778A0E1277886E1014084E2A3FFFFEAE4
:1004E0000D00A0E3EDFEFFEB2D00A0E3EBFEFFEB24
:1004F0002D00A0E3E9FEFFEB0D00A0E3E7FEFFEB1C
:100500000A00A0E3E5FEFFEB0A00A0E3E3FEFFEB39
:100510000209A0E3C6FEFFEB0A00A0E1F047BDE838
:100520001EFF2FE10800A0E100FFFFEB0040A0E369
:100530008EFFFFEA693829E02334A0E1FF3CC3E3E2
:10054000699423E00700A0E1088087E00910A0E19A
:10055000ADFEFFEB088089E0047087E20E40A0E367
:0805600082FFFFEA7856341215
:040000030000800079
:00000001FF
